:020000040000FA
:020000000428D2
:08000800FF30A200FF30A3004D
:10001000FF30A400FF30A5000F30A6008A110A129D
:100020003221AA108A110A123A21A6108A110A1244
:1000300055211E308A110A12452123108A110A12F5
:100040006D21A3108A110A126A2123118A110A1242
:100050006721A3118A110A12642123128A110A123C
:100060006121A3168A110A125E2123178A110A122E
:100070005B21A3178A110A12582100308A110A1233
:100080003D2100308A110A1270210F308A110A12A4
:10009000412100308A110A127421AB018A110A121F
:1000A000CC20EE308A110A129B2001308A110A12EC
:1000B000ED208A110A126B208A110A123D21AB0A27
:1000C0002B08FF3A8A110A1241218A110A124E287E
:1000D0008A110A1268288A110A12CC20AA308A11C1
:1000E0000A129B208A110A1276200800AC010830FF
:1000F000AD000310AC0CAA148A110A123A21013087
:100100008A110A122421AA108A110A123A210830EF
:100110008A110A122421AC138A110A12861E912810
:10012000AC1733308A110A1224218A110A12AD0B3E
:1001300079282C080800AC000830AD000310AC0C86
:100140008A110A12031CB728AA148A110A123A212A
:1001500001308A110A122421AA108A110A123A21A6
:100160003B308A110A1224218A110A12C328AA14C8
:100170008A110A123A213C308A110A122421AA104B
:100180008A110A123A2101308A110A1224218A1195
:100190000A12AD0B9E280800AA148A110A123A21ED
:1001A00030308A110A121021AA108A110A123A213B
:1001B00041308A110A122421A0118A110A12861ACA
:1001C000E228A0152A308A110A12102120118A1162
:1001D0000A12A01DEC2820150800AC002C08AD0068
:1001E0006430AE0064308A110A12F628AF00FF3086
:1001F000B0002E08B2002D08B10077308A110A1223
:100200003007031800298A110A12B10BFD288A1140
:100210000A12B20BFB288A110A12AF0BF928080048
:10022000AC002C08AD00AD088A110A12031D1B2971
:100230008A110A1223290A308A110A122421AD03D5
:100240008A110A1213290800AE00FE30AF00FF30F9
:10025000B0008A110A122E082F07031C0034300741
:100260002D2908008A110A128E2107309F008A1159
:100270000A1291298A110A124929A9008A110A121F
:100280004C29A8008A110A124F29A7008A110A12C4
:1002900052292A088900080029088800080028082F
:1002A000870008002708860008008A110A127829AA
:1002B0008A110A128B298A110A128B298A110A12B1
:1002C0008B298A110A128B298A110A128B298A1109
:1002D0000A128B298A110A128B298A110A128B2978
:1002E000A5008A110A128029A4008A110A128829FD
:1002F00026088A110A128E2189008A110A12912970
:1003000025088A110A128E2188008A110A12912961
:1003100024086700080023086600080083160313FA
:0803200008008312031308001A
:02400E00723FFF
:00000001FF
